 instrument

 Timestamp is ffffffff (Sun Feb  7 06:28:15 2106)

 Preferred load address is 10000000

 Start         Length     Name                   Class
 0001:00000000 000050a5H .text$mn                CODE
 0002:00000000 000000d8H .idata$5                DATA
 0002:000000d8 00000004H .00cfg                  DATA
 0002:000000dc 00000004H .CRT$XCA                DATA
 0002:000000e0 00000004H .CRT$XCZ                DATA
 0002:000000e4 00000004H .CRT$XIA                DATA
 0002:000000e8 00000004H .CRT$XIZ                DATA
 0002:000000ec 00000004H .CRT$XPA                DATA
 0002:000000f0 00000004H .CRT$XPZ                DATA
 0002:000000f4 00000004H .CRT$XTA                DATA
 0002:000000f8 00000008H .CRT$XTZ                DATA
 0002:000000fc 00000000H .gfids$y                DATA
 0002:00000100 000016c0H .rdata                  DATA
 0002:000017c0 00000004H .rdata$sxdata           DATA
 0002:000017c4 00000288H .rdata$zzzdbg           DATA
 0002:00001a4c 00000004H .rtc$IAA                DATA
 0002:00001a50 00000004H .rtc$IZZ                DATA
 0002:00001a54 00000004H .rtc$TAA                DATA
 0002:00001a58 00000008H .rtc$TZZ                DATA
 0002:00001a60 00000080H .xdata$x                DATA
 0002:00001ae0 00000418H .edata                  DATA
 0002:00001ef8 000000b4H .idata$2                DATA
 0002:00001fac 00000014H .idata$3                DATA
 0002:00001fc0 000000d8H .idata$4                DATA
 0002:00002098 0000041aH .idata$6                DATA
 0003:00000000 00000018H .data                   DATA
 0003:00000018 0000039cH .bss                    DATA
 0004:00000000 00000060H .rsrc$01                DATA
 0004:00000060 00000320H .rsrc$02                DATA

  Address         Publics by Value              Rva+Base       Lib:Object

 0000:00000000       ___hybrid_auxiliary_iat    00000000     <absolute>
 0000:00000000       ___volatile_metadata       00000000     <absolute>
 0000:00000000       ___guard_iat_table         00000000     <absolute>
 0000:00000000       ___enclave_config          00000000     <absolute>
 0000:00000000       ___dynamic_value_reloc_table 00000000     <absolute>
 0000:00000000       ___hybrid_code_map         00000000     <absolute>
 0000:00000000       ___guard_longjmp_count     00000000     <absolute>
 0000:00000000       ___guard_fids_count        00000000     <absolute>
 0000:00000000       ___guard_longjmp_table     00000000     <absolute>
 0000:00000000       ___hybrid_code_map_count   00000000     <absolute>
 0000:00000000       ___guard_fids_table        00000000     <absolute>
 0000:00000000       ___guard_iat_count         00000000     <absolute>
 0000:00000001       ___safe_se_handler_count   00000001     <absolute>
 0000:00000100       ___guard_flags             00000100     <absolute>
 0000:00000000       ___ImageBase               10000000     <linker-defined>
 0001:00000000       _convertUtf8ToModifiedUtf8 10001000 f   EncodingSupport.obj
 0001:0000011a       _modifiedUtf8LengthOfUtf8  1000111a f   EncodingSupport.obj
 0001:000001e0       _convertUft8ToPlatformString 100011e0 f   EncodingSupport_md.obj
 0001:000002c3       ___local_stdio_printf_options 100012c3 f i FileSystemSupport_md.obj
 0001:000002c9       __vfprintf_l               100012c9 f i FileSystemSupport_md.obj
 0001:000002ed       _basePath                  100012ed f   FileSystemSupport_md.obj
 0001:00000365       _fprintf                   10001365 f i FileSystemSupport_md.obj
 0001:0000037d       _fromURIPath               1000137d f   FileSystemSupport_md.obj
 0001:00000409       _isAbsolute                10001409 f   FileSystemSupport_md.obj
 0001:00000479       _normalize                 10001479 f   FileSystemSupport_md.obj
 0001:0000068f       _resolve                   1000168f f   FileSystemSupport_md.obj
 0001:000007b6       _Java_sun_instrument_InstrumentationImpl_appendToClassLoaderSearch0@24 100017b6 f   InstrumentationImplNativeMethods.obj
 0001:000007d1       _Java_sun_instrument_InstrumentationImpl_getAllLoadedClasses0@16 100017d1 f   InstrumentationImplNativeMethods.obj
 0001:000007e3       _Java_sun_instrument_InstrumentationImpl_getInitiatedClasses0@20 100017e3 f   InstrumentationImplNativeMethods.obj
 0001:000007fa       _Java_sun_instrument_InstrumentationImpl_getObjectSize0@20 100017fa f   InstrumentationImplNativeMethods.obj
 0001:00000811       _Java_sun_instrument_InstrumentationImpl_isModifiableClass0@20 10001811 f   InstrumentationImplNativeMethods.obj
 0001:00000828       _Java_sun_instrument_InstrumentationImpl_isRetransformClassesSupported0@16 10001828 f   InstrumentationImplNativeMethods.obj
 0001:0000083a       _Java_sun_instrument_InstrumentationImpl_loadAgent0@12 1000183a f   InstrumentationImplNativeMethods.obj
 0001:00000867       _Java_sun_instrument_InstrumentationImpl_redefineClasses0@20 10001867 f   InstrumentationImplNativeMethods.obj
 0001:0000087e       _Java_sun_instrument_InstrumentationImpl_retransformClasses0@20 1000187e f   InstrumentationImplNativeMethods.obj
 0001:00000895       _Java_sun_instrument_InstrumentationImpl_setHasRetransformableTransformers@20 10001895 f   InstrumentationImplNativeMethods.obj
 0001:000008ac       _Java_sun_instrument_InstrumentationImpl_setHasTransformers@20 100018ac f   InstrumentationImplNativeMethods.obj
 0001:000008c3       _Java_sun_instrument_InstrumentationImpl_setNativeMethodPrefixes@24 100018c3 f   InstrumentationImplNativeMethods.obj
 0001:000008de       _Agent_OnAttach@12         100018de f   InvocationAdapter.obj
 0001:00000bd1       _Agent_OnLoad@12           10001bd1 f   InvocationAdapter.obj
 0001:00000e16       _Agent_OnUnload@4          10001e16 f   InvocationAdapter.obj
 0001:0000118f       _convertCapabilityAttributes 1000218f f   InvocationAdapter.obj
 0001:00001359       _eventHandlerClassFileLoadHook@40 10002359 f   InvocationAdapter.obj
 0001:000013b1       _eventHandlerVMInit@12     100023b1 f   InvocationAdapter.obj
 0001:00001456       _getBooleanAttribute       10002456 f   InvocationAdapter.obj
 0001:00001481       _loadAgent                 10002481 f   InvocationAdapter.obj
 0001:00001736       _addNativeMethodPrefixCapability 10002736 f   JPLISAgent.obj
 0001:00001765       _addOriginalMethodOrderCapability 10002765 f   JPLISAgent.obj
 0001:000017ed       _addRedefineClassesCapability 100027ed f   JPLISAgent.obj
 0001:00001899       _allocateJPLISAgent        10002899 f   JPLISAgent.obj
 0001:000018a7       _appendToClassLoaderSearch 100028a7 f   JPLISAgent.obj
 0001:000019b2       _checkCapabilities         100029b2 f   JPLISAgent.obj
 0001:00001a37       _commandStringIntoJavaStrings 10002a37 f   JPLISAgent.obj
 0001:00001ae4       _commonGetClassList        10002ae4 f   JPLISAgent.obj
 0001:00001ba7       _createInstrumentationImpl 10002ba7 f   JPLISAgent.obj
 0001:00001e26       _createNewJPLISAgent       10002e26 f   JPLISAgent.obj
 0001:00001ebb       _deallocateCommandLineData 10002ebb f   JPLISAgent.obj
 0001:00001ee3       _enableNativeMethodPrefixCapability 10002ee3 f   JPLISAgent.obj
 0001:00001f65       _getAllLoadedClasses       10002f65 f   JPLISAgent.obj
 0001:00001f7d       _getAllLoadedClassesClassListFetcher 10002f7d f   JPLISAgent.obj
 0001:00001f93       _getInitiatedClasses       10002f93 f   JPLISAgent.obj
 0001:00001fad       _getInitiatedClassesClassListFetcher 10002fad f   JPLISAgent.obj
 0001:00001fc7       _getJPLISEnvironment       10002fc7 f   JPLISAgent.obj
 0001:00002113       _getObjectArrayFromClasses 10003113 f   JPLISAgent.obj
 0001:000021d3       _getObjectSize             100031d3 f   JPLISAgent.obj
 0001:0000224b       _initializeJPLISAgent      1000324b f   JPLISAgent.obj
 0001:000023b4       _invokeJavaAgentMainMethod 100033b4 f   JPLISAgent.obj
 0001:00002420       _isModifiableClass         10003420 f   JPLISAgent.obj
 0001:0000246b       _isRetransformClassesSupported 1000346b f   JPLISAgent.obj
 0001:00002473       _processJavaStart          10003473 f   JPLISAgent.obj
 0001:00002551       _recordCommandLineData     10003551 f   JPLISAgent.obj
 0001:000025ed       _redefineClassMapper       100035ed f   JPLISAgent.obj
 0001:0000269a       _redefineClasses           1000369a f   JPLISAgent.obj
 0001:00002b2a       _retransformClasses        10003b2a f   JPLISAgent.obj
 0001:00002cfc       _retransformableEnvironment 10003cfc f   JPLISAgent.obj
 0001:00002e90       _setHasRetransformableTransformers 10003e90 f   JPLISAgent.obj
 0001:00002ef8       _setHasTransformers        10003ef8 f   JPLISAgent.obj
 0001:00002f5a       _setLivePhaseEventHandlers 10003f5a f   JPLISAgent.obj
 0001:00002fff       _setNativeMethodPrefixes   10003fff f   JPLISAgent.obj
 0001:00003295       _startJavaAgent            10004295 f   JPLISAgent.obj
 0001:000032db       _transformClassFile        100042db f   JPLISAgent.obj
 0001:000035af       _JPLISAssertCondition      100045af f   JPLISAssert.obj
 0001:000035da       _JPLISAssertConditionWithMessage 100045da f   JPLISAssert.obj
 0001:000036b5       _freeAttributes            100046b5 f   JarFacade.obj
 0001:000036e2       _getAttribute              100046e2 f   JarFacade.obj
 0001:0000370b       _readAttributes            1000470b f   JarFacade.obj
 0001:0000373f       _checkForAndClearThrowable 1000473f f   JavaExceptions.obj
 0001:0000375f       _checkForThrowable         1000475f f   JavaExceptions.obj
 0001:0000376d       _createAndThrowInternalError 1000476d f   JavaExceptions.obj
 0001:0000378f       _createAndThrowThrowableFromJVMTIErrorCode 1000478f f   JavaExceptions.obj
 0001:000037b3       _createInternalError       100047b3 f   JavaExceptions.obj
 0001:000037c9       _createThrowable           100047c9 f   JavaExceptions.obj
 0001:000038f0       _createThrowableFromJVMTIErrorCode 100048f0 f   JavaExceptions.obj
 0001:00003a59       _getMessageFromThrowable   10004a59 f   JavaExceptions.obj
 0001:00003b62       _initializeFallbackError   10004b62 f   JavaExceptions.obj
 0001:00003bbf       _isSafeForJNICalls         10004bbf f   JavaExceptions.obj
 0001:00003bd3       _isUnchecked               10004bd3 f   JavaExceptions.obj
 0001:00003c60       _logThrowable              10004c60 f   JavaExceptions.obj
 0001:00003c78       _mapAllCheckedToInternalErrorMapper 10004c78 f   JavaExceptions.obj
 0001:00003d0f       _mapThrownThrowableIfNecessary 10004d0f f   JavaExceptions.obj
 0001:00003d4e       _preserveThrowable         10004d4e f   JavaExceptions.obj
 0001:00003d6b       _restoreThrowable          10004d6b f   JavaExceptions.obj
 0001:00003d70       _throwThrowable            10004d70 f   JavaExceptions.obj
 0001:0000407a       _validatePathChars         1000507a f   PathCharsValidator.obj
 0001:0000416a       _assertTLSValue            1000516a f   Reentrancy.obj
 0001:000041c9       _confirmingTLSSet          100051c9 f   Reentrancy.obj
 0001:000041fe       _releaseReentrancyToken    100051fe f   Reentrancy.obj
 0001:00004248       _tryToAcquireReentrancyToken 10005248 f   Reentrancy.obj
 0001:000042ea       _abortJVM                  100052ea f   Utilities.obj
 0001:000042f9       _allocate                  100052f9 f   Utilities.obj
 0001:00004343       _deallocate                10005343 f   Utilities.obj
 0001:00004377       _isInstanceofClassName     10005377 f   Utilities.obj
 0001:00004423       _Canonicalize              10005423 f   java:java.dll
 0001:00004429       _JLI_ManifestIterate@12    10005429 f   jli:jli.dll
 0001:0000442f       @__security_check_cookie@4 1000542f f   MSVCRT:secchk.obj
 0001:00004760       __DllMainCRTStartup@12     10005760 f   MSVCRT:dll_dllmain.obj
 0001:00004783       ___raise_securityfailure   10005783 f   MSVCRT:gs_report.obj
 0001:000047ab       ___report_gsfailure        100057ab f   MSVCRT:gs_report.obj
 0001:000048f1       ___security_init_cookie    100058f1 f   MSVCRT:gs_support.obj
 0001:0000493c       _DllMain@12                1000593c f   MSVCRT:dll_dllmain_stub.obj
 0001:0000495e       ?__scrt_initialize_type_info@@YAXXZ 1000595e f   MSVCRT:tncleanup.obj
 0001:0000496a       ?__scrt_uninitialize_type_info@@YAXXZ 1000596a f   MSVCRT:tncleanup.obj
 0001:00004976       ___local_stdio_scanf_options 10005976 f i MSVCRT:default_local_stdio_options.obj
 0001:0000497c       ___scrt_initialize_default_local_stdio_options 1000597c f   MSVCRT:default_local_stdio_options.obj
 0001:000049dd       ___scrt_acquire_startup_lock 100059dd f   MSVCRT:utility.obj
 0001:00004a0f       ___scrt_dllmain_after_initialize_c 10005a0f f   MSVCRT:utility.obj
 0001:00004a3a       ___scrt_dllmain_before_initialize_c 10005a3a f   MSVCRT:utility.obj
 0001:00004a48       ___scrt_dllmain_crt_thread_attach 10005a48 f   MSVCRT:utility.obj
 0001:00004a67       ___scrt_dllmain_crt_thread_detach 10005a67 f   MSVCRT:utility.obj
 0001:00004a74       ___scrt_dllmain_exception_filter 10005a74 f   MSVCRT:utility.obj
 0001:00004aa8       ___scrt_dllmain_uninitialize_c 10005aa8 f   MSVCRT:utility.obj
 0001:00004acb       ___scrt_dllmain_uninitialize_critical 10005acb f   MSVCRT:utility.obj
 0001:00004ad8       ___scrt_initialize_crt     10005ad8 f   MSVCRT:utility.obj
 0001:00004b11       ___scrt_initialize_onexit_tables 10005b11 f   MSVCRT:utility.obj
 0001:00004bb6       ___scrt_is_nonwritable_in_current_image 10005bb6 f   MSVCRT:utility.obj
 0001:00004c4a       ___scrt_release_startup_lock 10005c4a f   MSVCRT:utility.obj
 0001:00004c67       ___scrt_uninitialize_crt   10005c67 f   MSVCRT:utility.obj
 0001:00004c8f       ___scrt_get_dyn_tls_init_callback 10005c8f f   MSVCRT:dyn_tls_init.obj
 0001:00004c95       ___scrt_fastfail           10005c95 f   MSVCRT:utility_desktop.obj
 0001:00004daf       __crt_debugger_hook        10005daf f   MSVCRT:utility_desktop.obj
 0001:00004db7       __RTC_Initialize           10005db7 f   MSVCRT:initsect.obj
 0001:00004de3       __RTC_Terminate            10005de3 f   MSVCRT:initsect.obj
 0001:00004e10       __SEH_prolog4              10005e10 f   MSVCRT:sehprolg4.obj
 0001:00004e56       __SEH_epilog4              10005e56 f   MSVCRT:sehprolg4.obj
 0001:00004e6b       __except_handler4          10005e6b f   MSVCRT:chandler4gs.obj
 0001:00004e8e       @_guard_check_icall_nop@4  10005e8e f i MSVCRT:guard_support.obj
 0001:00004e92       ___isa_available_init      10005e92 f   MSVCRT:cpu_disp.obj
 0001:00005029       __get_startup_argv_mode    10006029 f   MSVCRT:argv_mode.obj
 0001:0000502d       ___scrt_is_ucrt_dll_in_use 1000602d f   MSVCRT:ucrt_detection.obj
 0001:00005039       _IsProcessorFeaturePresent@4 10006039 f   kernel32:KERNEL32.dll
 0001:0000503f       _memcpy                    1000603f f   vcruntime:VCRUNTIME140.dll
 0001:00005045       _strchr                    10006045 f   vcruntime:VCRUNTIME140.dll
 0001:0000504b       _memset                    1000604b f   vcruntime:VCRUNTIME140.dll
 0001:00005051       _strrchr                   10006051 f   vcruntime:VCRUNTIME140.dll
 0001:00005057       ___std_type_info_destroy_list 10006057 f   vcruntime:VCRUNTIME140.dll
 0001:0000505d       __except_handler4_common   1000605d f   vcruntime:VCRUNTIME140.dll
 0001:00005063       _strlen                    10006063 f   ucrt:api-ms-win-crt-string-l1-1-0.dll
 0001:00005069       _strcpy                    10006069 f   ucrt:api-ms-win-crt-string-l1-1-0.dll
 0001:0000506f       __initterm                 1000606f f   ucrt:api-ms-win-crt-runtime-l1-1-0.dll
 0001:00005075       __initterm_e               10006075 f   ucrt:api-ms-win-crt-runtime-l1-1-0.dll
 0001:0000507b       __seh_filter_dll           1000607b f   ucrt:api-ms-win-crt-runtime-l1-1-0.dll
 0001:00005081       __configure_narrow_argv    10006081 f   ucrt:api-ms-win-crt-runtime-l1-1-0.dll
 0001:00005087       __initialize_narrow_environment 10006087 f   ucrt:api-ms-win-crt-runtime-l1-1-0.dll
 0001:0000508d       __initialize_onexit_table  1000608d f   ucrt:api-ms-win-crt-runtime-l1-1-0.dll
 0001:00005093       __execute_onexit_table     10006093 f   ucrt:api-ms-win-crt-runtime-l1-1-0.dll
 0001:00005099       __cexit                    10006099 f   ucrt:api-ms-win-crt-runtime-l1-1-0.dll
 0001:0000509f       ___acrt_uninitialize_critical 1000609f f   MSVCRT:ucrt_stubs.obj
 0001:0000509f       ___acrt_thread_detach      1000609f f   MSVCRT:ucrt_stubs.obj
 0001:0000509f       ___scrt_stub_for_acrt_initialize 1000609f f   MSVCRT:ucrt_stubs.obj
 0001:0000509f       ___vcrt_thread_attach      1000609f f   MSVCRT:ucrt_stubs.obj
 0001:0000509f       ___acrt_uninitialize       1000609f f   MSVCRT:ucrt_stubs.obj
 0001:0000509f       ___scrt_stub_for_acrt_thread_attach 1000609f f   MSVCRT:ucrt_stubs.obj
 0001:0000509f       ___scrt_stub_for_acrt_uninitialize 1000609f f   MSVCRT:ucrt_stubs.obj
 0001:0000509f       ___vcrt_thread_detach      1000609f f   MSVCRT:ucrt_stubs.obj
 0001:0000509f       ___vcrt_initialize         1000609f f   MSVCRT:ucrt_stubs.obj
 0001:0000509f       ___acrt_thread_attach      1000609f f   MSVCRT:ucrt_stubs.obj
 0001:0000509f       ___acrt_initialize         1000609f f   MSVCRT:ucrt_stubs.obj
 0001:0000509f       ___vcrt_uninitialize_critical 1000609f f   MSVCRT:ucrt_stubs.obj
 0001:0000509f       ___scrt_stub_for_acrt_thread_detach 1000609f f   MSVCRT:ucrt_stubs.obj
 0001:0000509f       ___scrt_stub_for_acrt_uninitialize_critical 1000609f f   MSVCRT:ucrt_stubs.obj
 0001:0000509f       ___vcrt_uninitialize       1000609f f   MSVCRT:ucrt_stubs.obj
 0001:000050a2       ___scrt_stub_for_is_c_termination_complete 100060a2 f   MSVCRT:ucrt_stubs.obj
 0001:000050a2       __is_c_termination_complete 100060a2 f   MSVCRT:ucrt_stubs.obj
 0002:00000000       __imp__IsProcessorFeaturePresent@4 10007000     kernel32:KERNEL32.dll
 0002:00000004       __imp__IsDebuggerPresent@0 10007004     kernel32:KERNEL32.dll
 0002:00000008       __imp__MultiByteToWideChar@24 10007008     kernel32:KERNEL32.dll
 0002:0000000c       __imp__WideCharToMultiByte@32 1000700c     kernel32:KERNEL32.dll
 0002:00000010       __imp__GetACP@0            10007010     kernel32:KERNEL32.dll
 0002:00000014       __imp__GetLocaleInfoA@16   10007014     kernel32:KERNEL32.dll
 0002:00000018       __imp__GetUserDefaultLCID@0 10007018     kernel32:KERNEL32.dll
 0002:0000001c       __imp__UnhandledExceptionFilter@4 1000701c     kernel32:KERNEL32.dll
 0002:00000020       __imp__SetUnhandledExceptionFilter@4 10007020     kernel32:KERNEL32.dll
 0002:00000024       __imp__GetCurrentProcess@0 10007024     kernel32:KERNEL32.dll
 0002:00000028       __imp__TerminateProcess@8  10007028     kernel32:KERNEL32.dll
 0002:0000002c       __imp__DisableThreadLibraryCalls@4 1000702c     kernel32:KERNEL32.dll
 0002:00000030       __imp__QueryPerformanceCounter@4 10007030     kernel32:KERNEL32.dll
 0002:00000034       __imp__GetCurrentProcessId@0 10007034     kernel32:KERNEL32.dll
 0002:00000038       __imp__GetCurrentThreadId@0 10007038     kernel32:KERNEL32.dll
 0002:0000003c       __imp__GetSystemTimeAsFileTime@4 1000703c     kernel32:KERNEL32.dll
 0002:00000040       __imp__InitializeSListHead@4 10007040     kernel32:KERNEL32.dll
 0002:00000044       \177KERNEL32_NULL_THUNK_DATA 10007044     kernel32:KERNEL32.dll
 0002:00000048       __imp____std_type_info_destroy_list 10007048     vcruntime:VCRUNTIME140.dll
 0002:0000004c       __imp___except_handler4_common 1000704c     vcruntime:VCRUNTIME140.dll
 0002:00000050       __imp__memset              10007050     vcruntime:VCRUNTIME140.dll
 0002:00000054       __imp__memcpy              10007054     vcruntime:VCRUNTIME140.dll
 0002:00000058       __imp__strchr              10007058     vcruntime:VCRUNTIME140.dll
 0002:0000005c       __imp__strrchr             1000705c     vcruntime:VCRUNTIME140.dll
 0002:00000060       \177VCRUNTIME140_NULL_THUNK_DATA 10007060     vcruntime:VCRUNTIME140.dll
 0002:00000064       __imp__atoi                10007064     ucrt:api-ms-win-crt-convert-l1-1-0.dll
 0002:00000068       \177api-ms-win-crt-convert-l1-1-0_NULL_THUNK_DATA 10007068     ucrt:api-ms-win-crt-convert-l1-1-0.dll
 0002:0000006c       __imp__calloc              1000706c     ucrt:api-ms-win-crt-heap-l1-1-0.dll
 0002:00000070       __imp__realloc             10007070     ucrt:api-ms-win-crt-heap-l1-1-0.dll
 0002:00000074       __imp__free                10007074     ucrt:api-ms-win-crt-heap-l1-1-0.dll
 0002:00000078       __imp__malloc              10007078     ucrt:api-ms-win-crt-heap-l1-1-0.dll
 0002:0000007c       \177api-ms-win-crt-heap-l1-1-0_NULL_THUNK_DATA 1000707c     ucrt:api-ms-win-crt-heap-l1-1-0.dll
 0002:00000080       __imp___execute_onexit_table 10007080     ucrt:api-ms-win-crt-runtime-l1-1-0.dll
 0002:00000084       __imp___cexit              10007084     ucrt:api-ms-win-crt-runtime-l1-1-0.dll
 0002:00000088       __imp___initialize_narrow_environment 10007088     ucrt:api-ms-win-crt-runtime-l1-1-0.dll
 0002:0000008c       __imp___initterm           1000708c     ucrt:api-ms-win-crt-runtime-l1-1-0.dll
 0002:00000090       __imp___initterm_e         10007090     ucrt:api-ms-win-crt-runtime-l1-1-0.dll
 0002:00000094       __imp___seh_filter_dll     10007094     ucrt:api-ms-win-crt-runtime-l1-1-0.dll
 0002:00000098       __imp___configure_narrow_argv 10007098     ucrt:api-ms-win-crt-runtime-l1-1-0.dll
 0002:0000009c       __imp___initialize_onexit_table 1000709c     ucrt:api-ms-win-crt-runtime-l1-1-0.dll
 0002:000000a0       \177api-ms-win-crt-runtime-l1-1-0_NULL_THUNK_DATA 100070a0     ucrt:api-ms-win-crt-runtime-l1-1-0.dll
 0002:000000a4       __imp____acrt_iob_func     100070a4     ucrt:api-ms-win-crt-stdio-l1-1-0.dll
 0002:000000a8       __imp____stdio_common_vfprintf 100070a8     ucrt:api-ms-win-crt-stdio-l1-1-0.dll
 0002:000000ac       \177api-ms-win-crt-stdio-l1-1-0_NULL_THUNK_DATA 100070ac     ucrt:api-ms-win-crt-stdio-l1-1-0.dll
 0002:000000b0       __imp__strlen              100070b0     ucrt:api-ms-win-crt-string-l1-1-0.dll
 0002:000000b4       __imp__strcpy              100070b4     ucrt:api-ms-win-crt-string-l1-1-0.dll
 0002:000000b8       __imp__strncpy             100070b8     ucrt:api-ms-win-crt-string-l1-1-0.dll
 0002:000000bc       __imp__strdup              100070bc     ucrt:api-ms-win-crt-string-l1-1-0.dll
 0002:000000bc       __imp___strdup             100070bc     ucrt:api-ms-win-crt-string-l1-1-0.dll
 0002:000000c0       __imp__stricmp             100070c0     ucrt:api-ms-win-crt-string-l1-1-0.dll
 0002:000000c0       __imp___stricmp            100070c0     ucrt:api-ms-win-crt-string-l1-1-0.dll
 0002:000000c4       \177api-ms-win-crt-string-l1-1-0_NULL_THUNK_DATA 100070c4     ucrt:api-ms-win-crt-string-l1-1-0.dll
 0002:000000c8       __imp__Canonicalize        100070c8     java:java.dll
 0002:000000cc       \177java_NULL_THUNK_DATA   100070cc     java:java.dll
 0002:000000d0       __imp__JLI_ManifestIterate@12 100070d0     jli:jli.dll
 0002:000000d4       \177jli_NULL_THUNK_DATA    100070d4     jli:jli.dll
 0002:000000d8       ___guard_check_icall_fptr  100070d8     MSVCRT:guard_support.obj
 0002:000000dc       ___xc_a                    100070dc     MSVCRT:initializers.obj
 0002:000000e0       ___xc_z                    100070e0     MSVCRT:initializers.obj
 0002:000000e4       ___xi_a                    100070e4     MSVCRT:initializers.obj
 0002:000000e8       ___xi_z                    100070e8     MSVCRT:initializers.obj
 0002:000000ec       ___xp_a                    100070ec     MSVCRT:initializers.obj
 0002:000000f0       ___xp_z                    100070f0     MSVCRT:initializers.obj
 0002:000000f4       ___xt_a                    100070f4     MSVCRT:initializers.obj
 0002:000000f8       ___xt_z                    100070f8     MSVCRT:initializers.obj
 0002:00000100       ??_C@_0CK@PECNJIMP@OOM?5error?5in?5native?5tmp?5buffer?5@ 10007100     FileSystemSupport_md.obj
 0002:0000012c       ??_C@_04LOAJBDKD@true@     1000712c     InvocationAdapter.obj
 0002:00000134       ??_C@_0BF@MPBBPFEA@Can?9Redefine?9Classes@ 10007134     InvocationAdapter.obj
 0002:0000014c       ??_C@_0BI@DOGNCBOD@Can?9Retransform?9Classes@ 1000714c     InvocationAdapter.obj
 0002:00000164       ??_C@_0BN@GGMNHHCI@Can?9Set?9Native?9Method?9Prefix@ 10007164     InvocationAdapter.obj
 0002:00000184       ??_C@_0CD@ONCIGEJ@Can?9Maintain?9Original?9Method?9Or@ 10007184     InvocationAdapter.obj
 0002:000001a8       ??_C@_0CI@HNHEPCMG@?9javaagent?3?5memory?5allocation?5f@ 100071a8     InvocationAdapter.obj
 0002:000001d0       ??_C@_0DF@GEAEBGFM@Error?5opening?5zip?5file?5or?5JAR?5m@ 100071d0     InvocationAdapter.obj
 0002:00000208       ??_C@_0O@FJIJHIPN@Premain?9Class@ 10007208     InvocationAdapter.obj
 0002:00000218       ??_C@_0DH@NNDEJOON@Failed?5to?5find?5Premain?9Class?5ma@ 10007218     InvocationAdapter.obj
 0002:00000250       ??_C@_0CM@BAFHELIF@?9javaagent?3?5Premain?9Class?5value@ 10007250     InvocationAdapter.obj
 0002:0000027c       ??_C@_0CG@MGGAPOHH@?9javaagent?3?5memory?5allocation?5f@ 1000727c     InvocationAdapter.obj
 0002:000002a4       ??_C@_0BA@EEOHCMMC@Boot?9Class?9Path@ 100072a4     InvocationAdapter.obj
 0002:000002b4       ??_C@_0DO@FCLCEKPM@java?4lang?4instrument?1?9javaagent@ 100072b4     InvocationAdapter.obj
 0002:000002f8       ??_C@_0EJ@MNINEPDM@java?4lang?4instrument?1?9javaagent@ 100072f8     InvocationAdapter.obj
 0002:00000344       ??_C@_0DG@GEFLELM@java?4lang?4instrument?1?9javaagent@ 10007344     InvocationAdapter.obj
 0002:0000037c       ??_C@_0CI@DPANPEKD@?9javaagent?3?5agent?5class?5not?5spe@ 1000737c     InvocationAdapter.obj
 0002:000003a4       ??_C@_0DA@KPCNALNC@java?4lang?4instrument?1?9javaagent@ 100073a4     InvocationAdapter.obj
 0002:000003d8       ??_C@_0EF@HEMJBLDG@s?2src?2java?4instrument?2share?2nat@ 100073d8     InvocationAdapter.obj
 0002:00000420       ??_C@_0P@CKGKOICP@result?$DN?$DNJNI_OK@ 10007420     InvocationAdapter.obj
 0002:00000430       ??_C@_0DE@KGGELLFG@Error?5opening?5zip?5file?5or?5JAR?5m@ 10007430     InvocationAdapter.obj
 0002:00000464       ??_C@_0M@HHCNJNFE@Agent?9Class@ 10007464     InvocationAdapter.obj
 0002:00000470       ??_C@_0DH@DADPHJGN@Failed?5to?5find?5Agent?9Class?5mani@ 10007470     InvocationAdapter.obj
 0002:000004a8       ??_C@_0GG@HGIJBLPF@Unable?5to?5add?5?$CFs?5to?5system?5clas@ 100074a8     InvocationAdapter.obj
 0002:00000510       ??_C@_0BO@PHLNGFOC@Agent?9Class?5value?5is?5too?5big?6@ 10007510     InvocationAdapter.obj
 0002:00000530       ??_C@_07IPNMCAN@success@   10007530     InvocationAdapter.obj
 0002:00000538       ??_C@_0BI@FNNMMHD@Agent?5failed?5to?5start?$CB?6@ 10007538     InvocationAdapter.obj
 0002:00000550       ??_C@_0BF@JIBAFKML@Launcher?9Agent?9Class@ 10007550     InvocationAdapter.obj
 0002:00000568       ??_C@_0BL@ENCPOIKC@java?1lang?1OutOfMemoryError@ 10007568     InvocationAdapter.obj
 0002:00000583       ??_C@_00CNPNBAHC@@         10007583     InvocationAdapter.obj
 0002:00000588       ??_C@_0EC@FMFJIMAJ@processing?5of?5?9javaagent?5failed@ 10007588     InvocationAdapter.obj
 0002:000005d0       ??_C@_0JF@EOMLGCNE@Unable?5to?5add?5?$CFs?5to?5system?5clas@ 100075d0     InvocationAdapter.obj
 0002:00000668       ??_C@_0EH@PGNCMPLF@processing?5of?5?9javaagent?5failed@ 10007668     InvocationAdapter.obj
 0002:000006b0       ??_C@_0DJ@BIOAMFJP@processing?5of?5?9javaagent?5failed@ 100076b0     InvocationAdapter.obj
 0002:000006ec       ??_C@_01GBGANLPD@0@        100076ec     InvocationAdapter.obj
 0002:000006f0       ??_C@_0FE@GJAPONAI@System?5class?5loader?5does?5not?5de@ 100076f0     InvocationAdapter.obj
 0002:00000748       ??_C@_0EA@GNNEHPOG@Unexpected?5error?5?$CI?$CFd?$CJ?5returned?5@ 10007748     InvocationAdapter.obj
 0002:00000788       ??_C@_0BE@JIIENKGJ@path?5?$CB?$DN?5?$CIchar?$CK?$CJNULL@ 10007788     InvocationAdapter.obj
 0002:0000079c       ??_C@_0DJ@KAMKBHCJ@WARNING?3?5illegal?5character?5in?5B@ 1000779c     InvocationAdapter.obj
 0002:000007d8       ??_C@_0BL@EGNHKKEM@?$CIvoid?$CK?$CJpath?5?$CB?$DN?5?$CIvoid?$CK?$CJNULL@ 100077d8     InvocationAdapter.obj
 0002:000007f4       ??_C@_0CE@BMNGMKPL@WARNING?3?5unable?5to?5canonicalize@ 100077f4     InvocationAdapter.obj
 0002:00000818       ??_C@_0BG@LFGEPDCD@parent?5?$CB?$DN?5?$CIchar?$CK?$CJNULL@ 10007818     InvocationAdapter.obj
 0002:00000830       ??_C@_0DJ@BINIAAK@WARNING?3?5?$CFs?5not?5added?5to?5bootst@ 10007830     InvocationAdapter.obj
 0002:0000086c       ??_C@_0CC@HMBHOALF@Illegal?5argument?5or?5not?5JAR?5fil@ 1000786c     InvocationAdapter.obj
 0002:00000890       ??_C@_0BG@IPMFCDFJ@Unexpected?5error?3?5?$CFd?6@ 10007890     InvocationAdapter.obj
 0002:000008a8       ??_C@_0DO@NEGKBKCG@s?2src?2java?4instrument?2share?2nat@ 100078a8     JPLISAgent.obj
 0002:000008e8       ??_C@_0BP@JFPONFCF@jvmtierror?5?$DN?$DN?5JVMTI_ERROR_NONE@ 100078e8     JPLISAgent.obj
 0002:00000908       ??_C@_0BE@JEGDIMFH@environment?5?$CB?$DN?5NULL@ 10007908     JPLISAgent.obj
 0002:0000091c       ??_C@_0CD@EAGMGAOH@environment?9?$DOmJVMTIEnv?5?$DN?$DN?5jvmti@ 1000791c     JPLISAgent.obj
 0002:00000940       ??_C@_0BF@ENNAMHOI@fallback?5init?5failed@ 10007940     JPLISAgent.obj
 0002:00000958       ??_C@_06KJFADLGN@result@   10007958     JPLISAgent.obj
 0002:00000960       ??_C@_0CJ@MKNLGBML@instrumentation?5instance?5creati@ 10007960     JPLISAgent.obj
 0002:0000098c       ??_C@_0CJ@BCMDJAKB@setting?5of?5live?5phase?5VM?5handle@ 1000798c     JPLISAgent.obj
 0002:000009b8       ??_C@_0BP@DKNGPINN@agent?5load?1premain?5call?5failed@ 100079b8     JPLISAgent.obj
 0002:000009d8       ??_C@_0CD@FJABNFOF@sun?1instrument?1InstrumentationI@ 100079d8     JPLISAgent.obj
 0002:000009fc       ??_C@_0CJ@HOIGMIGF@find?5class?5on?5InstrumentationIm@ 100079fc     JPLISAgent.obj
 0002:00000a28       ??_C@_0BC@NFAEECCL@?$CBerrorOutstanding@ 10007a28     JPLISAgent.obj
 0002:00000a3c       ??_C@_06DNGMMBGB@?$CIJZZ?$CJV@ 10007a3c     JPLISAgent.obj
 0002:00000a44       ??_C@_06FALKBLGB@?$DMinit?$DO@ 10007a44     JPLISAgent.obj
 0002:00000a4c       ??_C@_0CP@DNJEEBBF@find?5constructor?5on?5Instrumenta@ 10007a4c     JPLISAgent.obj
 0002:00000a7c       ??_C@_0CP@HELLCCDH@call?5constructor?5on?5Instrumenta@ 10007a7c     JPLISAgent.obj
 0002:00000aac       ??_C@_0BN@KICHEFJM@copy?5local?5ref?5to?5global?5ref@ 10007aac     JPLISAgent.obj
 0002:00000acc       ??_C@_0CI@HEGLGDKJ@?$CILjava?1lang?1String?$DLLjava?1lang?1S@ 10007acc     JPLISAgent.obj
 0002:00000af4       ??_C@_0BI@MHLLCGNO@loadClassAndCallPremain@ 10007af4     JPLISAgent.obj
 0002:00000b0c       ??_C@_0CE@KECKFJKE@can?8t?5find?5premain?5invoker?5meth@ 10007b0c     JPLISAgent.obj
 0002:00000b30       ??_C@_0BK@JAOFMOJK@loadClassAndCallAgentmain@ 10007b30     JPLISAgent.obj
 0002:00000b4c       ??_C@_0CG@DOGNAPEF@can?8t?5find?5agentmain?5invoker?5me@ 10007b4c     JPLISAgent.obj
 0002:00000b78       ??_C@_0HE@BEDHLJCA@?$CILjava?1lang?1Module?$DLLjava?1lang?1C@ 10007b78     JPLISAgent.obj
 0002:00000bec       ??_C@_09IFONHNKG@transform@ 10007bec     JPLISAgent.obj
 0002:00000bf8       ??_C@_0BO@LKBEMJID@can?8t?5find?5transform?5methodID@ 10007bf8     JPLISAgent.obj
 0002:00000c18       ??_C@_0CE@NNNMFAHP@can?8t?5create?5class?5name?5java?5st@ 10007c18     JPLISAgent.obj
 0002:00000c3c       ??_C@_0CB@GCBHBCEC@can?8t?5create?5options?5java?5strin@ 10007c3c     JPLISAgent.obj
 0002:00000c60       ??_C@_0BK@OLJIPBJG@mainCallingMethod?5?$CB?$DN?5NULL@ 10007c60     JPLISAgent.obj
 0002:00000c80       ??_C@_0EK@NBNNLAGF@jvmtierror?5?$DN?$DN?5JVMTI_ERROR_NONE?5@ 10007c80     JPLISAgent.obj
 0002:00000ccc       ??_C@_0CC@NONNBMCM@error?5in?5the?5JVMTI?5GetNamedModu@ 10007ccc     JPLISAgent.obj
 0002:00000cf0       ??_C@_0BI@GCGOKABC@err?5?$DN?$DN?5JVMTI_ERROR_NONE@ 10007cf0     JPLISAgent.obj
 0002:00000d08       ??_C@_0BJ@OFPEOMG@can?8t?5create?5name?5string@ 10007d08     JPLISAgent.obj
 0002:00000d24       ??_C@_0BI@KDNOCEBM@can?8t?5create?5byte?5array@ 10007d24     JPLISAgent.obj
 0002:00000d3c       ??_C@_0BM@NODFBCMB@can?8t?5set?5byte?5array?5region@ 10007d3c     JPLISAgent.obj
 0002:00000d58       ??_C@_0CE@NCFBINFF@agent?9?$DOmInstrumentationImpl?5?$CB?$DN?5@ 10007d58     JPLISAgent.obj
 0002:00000d7c       ??_C@_0BK@GEFGBHIE@agent?9?$DOmTransform?5?$CB?$DN?5NULL@ 10007d7c     JPLISAgent.obj
 0002:00000d98       ??_C@_0BN@JDJGIEH@transform?5method?5call?5failed@ 10007d98     JPLISAgent.obj
 0002:00000db8       ??_C@_0BH@DDPAAIBF@can?8t?5get?5array?5length@ 10007db8     JPLISAgent.obj
 0002:00000dd0       ??_C@_0BN@KNPJDEBO@can?8t?5allocate?5result?5buffer@ 10007dd0     JPLISAgent.obj
 0002:00000df0       ??_C@_0BM@CLGDMLIA@can?8t?5get?5byte?5array?5region@ 10007df0     JPLISAgent.obj
 0002:00000e0c       ??_C@_0BK@JCFBFKNG@isSafeForJNICalls?$CIjnienv?$CJ@ 10007e0c     JPLISAgent.obj
 0002:00000e28       ??_C@_0CF@PBJJFPHF@?$CBisUnchecked?$CIjnienv?0?5throwableT@ 10007e28     JPLISAgent.obj
 0002:00000e50       ??_C@_0CB@KCPANAMN@java?1lang?1ClassNotFoundExceptio@ 10007e50     JPLISAgent.obj
 0002:00000e74       ??_C@_0DA@MJOAEAPC@java?1lang?1instrument?1Unmodifiab@ 10007e74     JPLISAgent.obj
 0002:00000ea4       ??_C@_0BA@JJLOPNCP@java?1lang?1Class@ 10007ea4     JPLISAgent.obj
 0002:00000eb4       ??_C@_0BO@GBLMHFAI@FindClass?5returned?5null?5class@ 10007eb4     JPLISAgent.obj
 0002:00000ed4       ??_C@_0BI@JLMJJPLE@classArrayClass?5?$CB?$DN?5NULL@ 10007ed4     JPLISAgent.obj
 0002:00000eec       ??_C@_0CD@NMCFBNHK@NewObjectArray?5returned?5null?5ar@ 10007eec     JPLISAgent.obj
 0002:00000f10       ??_C@_0BD@BNJLEHDL@localArray?5?$CB?$DN?5NULL@ 10007f10     JPLISAgent.obj
 0002:00000f24       ??_C@_0CI@MJAJKCDF@jvmtierror?5?$DN?$DN?5JVMTI_ERROR_NOT_A@ 10007f24     JPLISAgent.obj
 0002:00000f4c       ??_C@_0BB@DBNGJIMM@jvmtienv?5?$CB?$DN?5NULL@ 10007f4c     JPLISAgent.obj
 0002:00000f60       ??_C@_0BJ@EJCHPAPK@retransformerEnv?5?$CB?$DN?5NULL@ 10007f60     JPLISAgent.obj
 0002:00000f7c       ??_C@_0BA@DKKKAEPC@classes?5?$CB?$DN?5NULL@ 10007f7c     JPLISAgent.obj
 0002:00000f8c       ??_C@_0P@IBHCMEIB@?$CBerrorOccurred@ 10007f8c     JPLISAgent.obj
 0002:00000f9c       ??_C@_0BA@DHKCDHMI@numClasses?5?$CB?$DN?50@ 10007f9c     JPLISAgent.obj
 0002:00000fac       ??_C@_0BK@HBLAKIEB@classArray?$FLindex?$FN?5?$CB?$DN?5NULL@ 10007fac     JPLISAgent.obj
 0002:00000fc8       ??_C@_0BJ@NGKAGHPG@classDefinitions?5?$CB?$DN?5NULL@ 10007fc8     JPLISAgent.obj
 0002:00000fe4       ??_C@_0M@KGLONNBG@numDefs?5?$DO?50@ 10007fe4     JPLISAgent.obj
 0002:00000ff0       ??_C@_0CF@BGAIILOJ@java?1lang?1instrument?1ClassDefin@ 10007ff0     JPLISAgent.obj
 0002:00001018       ??_C@_0BE@IIFEGCLG@?$CI?$CJLjava?1lang?1Class?$DL@ 10008018     JPLISAgent.obj
 0002:0000102c       ??_C@_0BD@FFKMDMBN@getDefinitionClass@ 1000802c     JPLISAgent.obj
 0002:00001040       ??_C@_04LHPAGAEF@?$CI?$CJ?$FLB@ 10008040     JPLISAgent.obj
 0002:00001048       ??_C@_0BH@FOGLHNOO@getDefinitionClassFile@ 10008048     JPLISAgent.obj
 0002:00001060       ??_C@_0BE@NLJNCPBN@prefixArray?5?$CB?$DN?5NULL@ 10008060     JPLISAgent.obj
 0002:00001078       ??_C@_0EE@FPMMKFJK@?$CK?$CK?$CK?5java?4lang?4instrument?5ASSERT@ 10008078     JPLISAssert.obj
 0002:000010c0       ??_C@_0FE@HCMNEDKA@?$CK?$CK?$CK?5java?4lang?4instrument?5ASSERT@ 100080c0     JPLISAssert.obj
 0002:00001118       ??_C@_0EC@BMPNKMFA@s?2src?2java?4instrument?2share?2nat@ 10008118     JavaExceptions.obj
 0002:0000115c       ??_C@_0BH@EKGMOCH@throwableToMap?5?$CB?$DN?5NULL@ 1000815c     JavaExceptions.obj
 0002:00001174       ??_C@_0BC@HKCJMFCP@className?5?$CB?$DN?5NULL@ 10008174     JavaExceptions.obj
 0002:00001188       ??_C@_0BG@IKDDPPGD@?$CILjava?1lang?1String?$DL?$CJV@ 10008188     JavaExceptions.obj
 0002:000011a0       ??_C@_0BI@NBLNIHIB@java?1lang?1InternalError@ 100081a0     JavaExceptions.obj
 0002:000011b8       ??_C@_0BP@GJLHLAKJ@java?1lang?1NullPointerException@ 100081b8     JavaExceptions.obj
 0002:000011d8       ??_C@_0CD@MOHADDFA@java?1lang?1IllegalArgumentExcept@ 100081d8     JavaExceptions.obj
 0002:000011fc       ??_C@_0CA@OCDKFHGJ@java?1lang?1ClassCircularityError@ 100081fc     JavaExceptions.obj
 0002:0000121c       ??_C@_0BG@FNCILCAN@java?1lang?1VerifyError@ 1000821c     JavaExceptions.obj
 0002:00001234       ??_C@_0CI@LDDEGNGM@java?1lang?1UnsupportedOperationE@ 10008234     JavaExceptions.obj
 0002:0000125c       ??_C@_0DF@IFGMNJBO@class?5redefinition?5failed?3?5atte@ 1000825c     JavaExceptions.obj
 0002:00001298       ??_C@_0EO@LOHFEPOO@class?5redefinition?5failed?3?5atte@ 10008298     JavaExceptions.obj
 0002:000012e8       ??_C@_0EI@PJGIIEAK@class?5redefinition?5failed?3?5atte@ 100082e8     JavaExceptions.obj
 0002:00001330       ??_C@_0DI@KJLEIONK@class?5redefinition?5failed?3?5atte@ 10008330     JavaExceptions.obj
 0002:00001368       ??_C@_0ED@PPHPPFFE@class?5redefinition?5failed?3?5atte@ 10008368     JavaExceptions.obj
 0002:000013b0       ??_C@_0FL@JFPGFPBC@class?5redefinition?5failed?3?5atte@ 100083b0     JavaExceptions.obj
 0002:00001410       ??_C@_0EA@INKOHMMN@class?5redefinition?5failed?3?5atte@ 10008410     JavaExceptions.obj
 0002:00001450       ??_C@_0CH@DNCLOIOF@java?1lang?1UnsupportedClassVersi@ 10008450     JavaExceptions.obj
 0002:00001478       ??_C@_0BP@NAHGIHIH@java?1lang?1NoClassDefFoundError@ 10008478     JavaExceptions.obj
 0002:00001498       ??_C@_0BI@MAPDCENK@class?5names?5don?8t?5match@ 10008498     JavaExceptions.obj
 0002:000014b0       ??_C@_0BL@EEAIAIEG@java?1lang?1ClassFormatError@ 100084b0     JavaExceptions.obj
 0002:000014cc       ??_C@_0CJ@DNCKJBBE@class?5redefinition?5failed?3?5inva@ 100084cc     JavaExceptions.obj
 0002:000014f8       ??_C@_0BG@JKFIFBMN@unsupported?5operation@ 100084f8     JavaExceptions.obj
 0002:00001510       ??_C@_0CD@LAOKENHO@can?8t?5create?5exception?5java?5str@ 10008510     JavaExceptions.obj
 0002:00001534       ??_C@_0BF@FOHFOJOB@?$CI?$CJLjava?1lang?1String?$DL@ 10008534     JavaExceptions.obj
 0002:0000154c       ??_C@_08JCDFGHAO@toString@ 1000854c     JavaExceptions.obj
 0002:00001558       ??_C@_0BA@NOLMKEPF@java?1lang?1Error@ 10008558     JavaExceptions.obj
 0002:00001568       ??_C@_0BL@IONOAEOO@java?1lang?1RuntimeException@ 10008568     JavaExceptions.obj
 0002:00001584       ??_C@_0CC@GKBBLNKJ@throwThrowable?5failed?5to?5re?9thr@ 10008584     JavaExceptions.obj
 0002:000015a8       ??_C@_0BB@EJBOEPOM@result?5?$DN?$DN?5JNI_OK@ 100085a8     JavaExceptions.obj
 0002:000015bc       ??_C@_09HLKPJHCC@?9_?4?$CB?$HO?$CK?8?$CI?$CJ@ 100085bc     PathCharsValidator.obj
 0002:000015c8       ??_C@_07DDNJCNOL@?3?$EA?$CG?$DN?$CL$?0@ 100085c8     PathCharsValidator.obj
 0002:000015d0       ??_C@_02DKJMBEPB@?$DL?1@   100085d0     PathCharsValidator.obj
 0002:000015d4       ??_C@_0DO@IILOFBP@s?2src?2java?4instrument?2share?2nat@ 100085d4     Reentrancy.obj
 0002:00001614       ??_C@_0BK@PPCACBKK@error?5?$DN?$DN?5JVMTI_ERROR_NONE@ 10008614     Reentrancy.obj
 0002:00001630       ??_C@_0BB@LLFPNPAC@test?5?$DN?$DN?5expected@ 10008630     Reentrancy.obj
 0002:00001644       ??_C@_0DN@HOJJMEHN@s?2src?2java?4instrument?2share?2nat@ 10008644     Utilities.obj
 0002:00001684       ??_C@_0BI@NNKHJJFO@Can?8t?5deallocate?5memory@ 10008684     Utilities.obj
 0002:0000169c       __pDefaultRawDllMain       1000869c     MSVCRT:dll_dllmain.obj
 0002:0000169c       __pRawDllMain              1000869c     MSVCRT:dll_dllmain.obj
 0002:00001720       __load_config_used         10008720     MSVCRT:loadcfg.obj
 0002:000017c0       ___safe_se_handler_table   100087c0     <linker-defined>
 0002:00001a4c       ___rtc_iaa                 10008a4c     MSVCRT:initsect.obj
 0002:00001a50       ___rtc_izz                 10008a50     MSVCRT:initsect.obj
 0002:00001a54       ___rtc_taa                 10008a54     MSVCRT:initsect.obj
 0002:00001a58       ___rtc_tzz                 10008a58     MSVCRT:initsect.obj
 0002:00001ef8       __IMPORT_DESCRIPTOR_java   10008ef8     java:java.dll
 0002:00001f0c       __IMPORT_DESCRIPTOR_jli    10008f0c     jli:jli.dll
 0002:00001f20       __IMPORT_DESCRIPTOR_KERNEL32 10008f20     kernel32:KERNEL32.dll
 0002:00001f34       __IMPORT_DESCRIPTOR_VCRUNTIME140 10008f34     vcruntime:VCRUNTIME140.dll
 0002:00001f48       __IMPORT_DESCRIPTOR_api-ms-win-crt-heap-l1-1-0 10008f48     ucrt:api-ms-win-crt-heap-l1-1-0.dll
 0002:00001f5c       __IMPORT_DESCRIPTOR_api-ms-win-crt-convert-l1-1-0 10008f5c     ucrt:api-ms-win-crt-convert-l1-1-0.dll
 0002:00001f70       __IMPORT_DESCRIPTOR_api-ms-win-crt-stdio-l1-1-0 10008f70     ucrt:api-ms-win-crt-stdio-l1-1-0.dll
 0002:00001f84       __IMPORT_DESCRIPTOR_api-ms-win-crt-string-l1-1-0 10008f84     ucrt:api-ms-win-crt-string-l1-1-0.dll
 0002:00001f98       __IMPORT_DESCRIPTOR_api-ms-win-crt-runtime-l1-1-0 10008f98     ucrt:api-ms-win-crt-runtime-l1-1-0.dll
 0002:00001fac       __NULL_IMPORT_DESCRIPTOR   10008fac     java:java.dll
 0003:00000000       ___security_cookie_complement 1000a000     MSVCRT:gs_cookie.obj
 0003:00000004       ___security_cookie         1000a004     MSVCRT:gs_cookie.obj
 0003:00000008       ___scrt_native_dllmain_reason 1000a008     MSVCRT:utility.obj
 0003:00000010       ___isa_enabled             1000a010     MSVCRT:cpu_disp.obj
 0003:00000014       ___scrt_ucrt_dll_is_in_use 1000a014     MSVCRT:ucrt_stubs.obj
 0003:00000368       ?__type_info_root_node@@3U__type_info_node@@A 1000a368     MSVCRT:tncleanup.obj
 0003:00000370       ?_OptionsStorage@?1??__local_stdio_scanf_options@@9@4_KA 1000a370     MSVCRT:default_local_stdio_options.obj
 0003:00000378       ___scrt_current_native_startup_state 1000a378     MSVCRT:utility.obj
 0003:0000037c       ___scrt_native_startup_lock 1000a37c     MSVCRT:utility.obj
 0003:0000039c       ___scrt_debugger_hook_flag 1000a39c     MSVCRT:utility_desktop.obj
 0003:000003a0       ___isa_available           1000a3a0     MSVCRT:cpu_disp.obj
 0003:000003a4       ___favor                   1000a3a4     MSVCRT:cpu_disp.obj
 0003:000003a8       ?_OptionsStorage@?1??__local_stdio_printf_options@@9@9 1000a3a8     <common>
 0003:000003b0       ___dyn_tls_init_callback   1000a3b0     <common>

 entry point at        0001:00004760

 Static symbols

 0000:ffff3000       .debug$S                   10000000     kernel32:KERNEL32.dll
 0000:ffff3000       .debug$S                   10000000     java:java.dll
 0000:ffff3000       .debug$S                   10000000     jli:jli.dll
 0000:ffff3000       .debug$S                   10000000     kernel32:KERNEL32.dll
 0000:ffff3000       .debug$S                   10000000     kernel32:KERNEL32.dll
 0000:ffff3000       .debug$S                   10000000     kernel32:KERNEL32.dll
 0000:ffff3000       .debug$S                   10000000     kernel32:KERNEL32.dll
 0000:ffff3000       .debug$S                   10000000     kernel32:KERNEL32.dll
 0000:ffff3000       .debug$S                   10000000     kernel32:KERNEL32.dll
 0000:ffff3000       .debug$S                   10000000     kernel32:KERNEL32.dll
 0000:ffff3000       .debug$S                   10000000     kernel32:KERNEL32.dll
 0000:ffff3000       .debug$S                   10000000     kernel32:KERNEL32.dll
 0000:ffff3000       .debug$S                   10000000     kernel32:KERNEL32.dll
 0000:ffff3000       .debug$S                   10000000     kernel32:KERNEL32.dll
 0000:ffff3000       .debug$S                   10000000     kernel32:KERNEL32.dll
 0000:ffff3000       .debug$S                   10000000     kernel32:KERNEL32.dll
 0000:ffff3000       .debug$S                   10000000     kernel32:KERNEL32.dll
 0000:ffff3000       .debug$S                   10000000     kernel32:KERNEL32.dll
 0000:ffff3000       .debug$S                   10000000     kernel32:KERNEL32.dll
 0000:ffff3000       .debug$S                   10000000     vcruntime:VCRUNTIME140.dll
 0000:ffff3000       .debug$S                   10000000     instrument.exp
 0000:ffff3000       .debug$S                   10000000     kernel32:KERNEL32.dll
 0000:ffff3000       .debug$S                   10000000     kernel32:KERNEL32.dll
 0000:ffff3000       .debug$S                   10000000     vcruntime:VCRUNTIME140.dll
 0000:ffff3000       .debug$S                   10000000     vcruntime:VCRUNTIME140.dll
 0000:ffff3000       .debug$S                   10000000     vcruntime:VCRUNTIME140.dll
 0000:ffff3000       .debug$S                   10000000     vcruntime:VCRUNTIME140.dll
 0000:ffff3000       .debug$S                   10000000     ucrt:api-ms-win-crt-string-l1-1-0.dll
 0000:ffff3000       .debug$S                   10000000     ucrt:api-ms-win-crt-string-l1-1-0.dll
 0000:ffff3000       .debug$S                   10000000     ucrt:api-ms-win-crt-runtime-l1-1-0.dll
 0000:ffff3000       .debug$S                   10000000     ucrt:api-ms-win-crt-runtime-l1-1-0.dll
 0000:ffff3000       .debug$S                   10000000     ucrt:api-ms-win-crt-runtime-l1-1-0.dll
 0000:ffff3000       .debug$S                   10000000     ucrt:api-ms-win-crt-runtime-l1-1-0.dll
 0000:ffff3000       .debug$S                   10000000     ucrt:api-ms-win-crt-runtime-l1-1-0.dll
 0000:ffff3000       .debug$S                   10000000     ucrt:api-ms-win-crt-runtime-l1-1-0.dll
 0000:ffff3000       .debug$S                   10000000     ucrt:api-ms-win-crt-runtime-l1-1-0.dll
 0000:ffff3000       .debug$S                   10000000     ucrt:api-ms-win-crt-runtime-l1-1-0.dll
 0000:ffff3000       .debug$S                   10000000     ucrt:api-ms-win-crt-runtime-l1-1-0.dll
 0000:ffff3000       .debug$S                   10000000     ucrt:api-ms-win-crt-runtime-l1-1-0.dll
 0000:ffff3000       .debug$S                   10000000     ucrt:api-ms-win-crt-runtime-l1-1-0.dll
 0000:ffff3000       .debug$S                   10000000     ucrt:api-ms-win-crt-runtime-l1-1-0.dll
 0000:ffff3000       .debug$S                   10000000     ucrt:api-ms-win-crt-string-l1-1-0.dll
 0000:ffff3000       .debug$S                   10000000     ucrt:api-ms-win-crt-heap-l1-1-0.dll
 0000:ffff3000       .debug$S                   10000000     ucrt:api-ms-win-crt-heap-l1-1-0.dll
 0000:ffff3000       .debug$S                   10000000     ucrt:api-ms-win-crt-string-l1-1-0.dll
 0000:ffff3000       .debug$S                   10000000     ucrt:api-ms-win-crt-string-l1-1-0.dll
 0000:ffff3000       .debug$S                   10000000     ucrt:api-ms-win-crt-stdio-l1-1-0.dll
 0000:ffff3000       .debug$S                   10000000     ucrt:api-ms-win-crt-stdio-l1-1-0.dll
 0000:ffff3000       .debug$S                   10000000     ucrt:api-ms-win-crt-convert-l1-1-0.dll
 0000:ffff3000       .debug$S                   10000000     ucrt:api-ms-win-crt-heap-l1-1-0.dll
 0000:ffff3000       .debug$S                   10000000     ucrt:api-ms-win-crt-heap-l1-1-0.dll
 0000:ffff3000       .debug$S                   10000000     vcruntime:VCRUNTIME140.dll
 0001:00000466       _isSlash                   10001466 f   FileSystemSupport_md.obj
 0001:000004e5       _normalizePath             100014e5 f   FileSystemSupport_md.obj
 0001:000005eb       _normalizePrefix           100015eb f   FileSystemSupport_md.obj
 0001:00000e19       _appendBootClassPath       10001e19 f   InvocationAdapter.obj
 0001:00001132       _appendClassPath           10002132 f   InvocationAdapter.obj
 0001:00001204       _decodeNibble              10002204 f   InvocationAdapter.obj
 0001:00001236       _decodePath                10002236 f   InvocationAdapter.obj
 0001:0000161b       _parseArgumentTail         1000261b f   InvocationAdapter.obj
 0001:000016b3       _splitPathList             100026b3 f   InvocationAdapter.obj
 0001:00002052       _getModuleObject           10003052 f   JPLISAgent.obj
 0001:00003608       _doAttribute               10004608 f   JarFacade.obj
 0001:00003dab       _highMask                  10004dab f   PathCharsValidator.obj
 0001:00003e11       _highMaskRange             10004e11 f   PathCharsValidator.obj
 0001:00003e89       _initialize                10004e89 f   PathCharsValidator.obj
 0001:00003fb2       _lowMask                   10004fb2 f   PathCharsValidator.obj
 0001:00004010       _match                     10005010 f   PathCharsValidator.obj
 0001:00004440       ?dllmain_crt_dispatch@@YGHQAUHINSTANCE__@@KQAX@Z 10005440 f   MSVCRT:dll_dllmain.obj
 0001:00004493       ?dllmain_crt_process_attach@@YAHQAUHINSTANCE__@@QAX@Z 10005493 f   MSVCRT:dll_dllmain.obj
 0001:0000459d       ?dllmain_crt_process_detach@@YAH_N@Z 1000559d f   MSVCRT:dll_dllmain.obj
 0001:0000462f       ?dllmain_dispatch@@YAHQAUHINSTANCE__@@KQAX@Z 1000562f f   MSVCRT:dll_dllmain.obj
 0001:00004735       ?dllmain_raw@@YGHQAUHINSTANCE__@@KQAX@Z 10005735 f   MSVCRT:dll_dllmain.obj
 0001:000048a4       ___get_entropy             100058a4 f   MSVCRT:gs_support.obj
 0001:00004999       ?find_pe_section@@YAPAU_IMAGE_SECTION_HEADER@@QAEI@Z 10005999 f   MSVCRT:utility.obj
 0001:00004e10       $$000000                   10005e10     MSVCRT:sehprolg4.obj
 0002:000016a0       _GS_ExceptionPointers      100086a0     MSVCRT:gs_report.obj
 0002:00001a60       __sehtable$?dllmain_crt_process_attach@@YAHQAUHINSTANCE__@@QAX@Z 10008a60     MSVCRT:dll_dllmain.obj
 0002:00001a80       __sehtable$?dllmain_crt_process_detach@@YAH_N@Z 10008a80     MSVCRT:dll_dllmain.obj
 0002:00001aa0       __sehtable$?dllmain_dispatch@@YAHQAUHINSTANCE__@@KQAX@Z 10008aa0     MSVCRT:dll_dllmain.obj
 0002:00001ac0       __sehtable$___scrt_is_nonwritable_in_current_image 10008ac0     MSVCRT:utility.obj
 0002:00001ae0       .edata                     10008ae0     instrument.exp
 0002:00001b08       rgpv                       10008b08     instrument.exp
 0002:00001b44       rgszName                   10008b44     instrument.exp
 0002:00001b80       rgwOrd                     10008b80     instrument.exp
 0002:00001b9e       szName                     10008b9e     instrument.exp
 0002:00001bad       $N00001                    10008bad     instrument.exp
 0002:00001bc0       $N00002                    10008bc0     instrument.exp
 0002:00001bd1       $N00003                    10008bd1     instrument.exp
 0002:00001be3       $N00004                    10008be3     instrument.exp
 0002:00001c2a       $N00005                    10008c2a     instrument.exp
 0002:00001c6b       $N00006                    10008c6b     instrument.exp
 0002:00001cac       $N00007                    10008cac     instrument.exp
 0002:00001ce7       $N00008                    10008ce7     instrument.exp
 0002:00001d26       $N00009                    10008d26     instrument.exp
 0002:00001d71       $N00010                    10008d71     instrument.exp
 0002:00001da8       $N00011                    10008da8     instrument.exp
 0002:00001de5       $N00012                    10008de5     instrument.exp
 0002:00001e25       $N00013                    10008e25     instrument.exp
 0002:00001e73       $N00014                    10008e73     instrument.exp
 0002:00001eb2       $N00015                    10008eb2     instrument.exp
 0002:000020a8       .idata$6                   100090a8     java:java.dll
 0002:000020cc       .idata$6                   100090cc     jli:jli.dll
 0002:00002256       .idata$6                   10009256     kernel32:KERNEL32.dll
 0002:000022c6       .idata$6                   100092c6     vcruntime:VCRUNTIME140.dll
 0002:0000240c       .idata$6                   1000940c     ucrt:api-ms-win-crt-heap-l1-1-0.dll
 0002:0000242c       .idata$6                   1000942c     ucrt:api-ms-win-crt-convert-l1-1-0.dll
 0002:0000244e       .idata$6                   1000944e     ucrt:api-ms-win-crt-stdio-l1-1-0.dll
 0002:0000246e       .idata$6                   1000946e     ucrt:api-ms-win-crt-string-l1-1-0.dll
 0002:00002490       .idata$6                   10009490     ucrt:api-ms-win-crt-runtime-l1-1-0.dll
 0003:00000018       _sFallbackInternalError    1000a018     JavaExceptions.obj
 0003:00000020       _L_HEX                     1000a020     PathCharsValidator.obj
 0003:00000028       _H_HEX                     1000a028     PathCharsValidator.obj
 0003:00000030       _L_PATH                    1000a030     PathCharsValidator.obj
 0003:00000038       _H_PATH                    1000a038     PathCharsValidator.obj
 0003:00000040       ?__proc_attached@@3HA      1000a040     MSVCRT:dll_dllmain.obj
 0003:00000048       _GS_ExceptionRecord        1000a048     MSVCRT:gs_report.obj
 0003:00000098       _GS_ContextRecord          1000a098     MSVCRT:gs_report.obj
 0003:00000380       ?is_initialized_as_dll@@3_NA 1000a380     MSVCRT:utility.obj
 0003:00000381       ?module_local_atexit_table_initialized@@3_NA 1000a381     MSVCRT:utility.obj
 0003:00000384       ?module_local_atexit_table@@3U_onexit_table_t@@A 1000a384     MSVCRT:utility.obj
 0003:00000390       ?module_local_at_quick_exit_table@@3U_onexit_table_t@@A 1000a390     MSVCRT:utility.obj
 0004:00000060       $R000000                   1000b060     instrument.dll.res
